S0220000687474703A2F2F737265636F72642E736F75726365666F7267652E6E65742F1D
S12300000C9438000C947A160C942F1E0C945F000C945F000C945F000C945F000C945F00EC
S12300200C945F000C94F21E0C945F000C94F6220C945F000C945B170C9435170C940B1698
S12300400C94F6230C945F000C9475230C945F000C949B240C9463240C945F000C945F0029
S12300600C945F000C945F000C945F000C945F0011241FBECFEFD0E1DEBFCDBF14BEA895C7
S123008088E10FB6F89480936000109260000FBE15E0A0E0B1E0E0EBFCE402C005900D92B9
S12300A0AE31B107D9F716E0AEE1B5E001C01D92AB3CB107E1F70E94750E0C9457260C94F2
S12300C0000020E030E0D901AC54BF4F0E943926802DF901EE5BFE4F80832F5F3F4F203A6D
S12300E0310589F720E030E0D901A857BE4F0E943926802DF901E55CFE4F80832F5F3F4FFB
S12301002530310589F712BC11BC089520E030E0F901EE5BFE4F8081D901AC54BF4F082ED9
S12301200E9446262F5F3F4F203A310589F712BC11BC08954E9B11C020E030E0D9015096BF
S12301400E943926802DF901EE51FE4F80832F5F3F4F203A310591F0F1CF20E030E0D9018D
S1230160A859BD4F0E943926802DF901EE51FE4F80832F5F3F4F203A310589F712BC11BC70
S123018008954E9B11C020E030E0F901EE51FE4F8081D9015096082E0E9446262F5F3F4F4D
S12301A0203A310591F0F1CF20E030E0F901EE51FE4F8081D901A859BD4F082E0E944626A8
S12301C02F5F3F4F203A310589F712BC11BC089520E931E0D9010E943926802D205531402F
S12301E0F901EE57FD4F80832F5A3E4F81E0203F380781F712BC11BC089520E430E0F9019A
S1230200EE57FD4F8081D901A05BBE4F082E0E9446262F5F3F4F203A310589F712BC11BC5B
S12302200895A2E0B0E00E943926802D90E090931F0180931E0120911E0130911F01A3E044
S1230240B0E00E943926802D90E0982F8827820F931F90931F0180931E01A4E0B0E00E9408
S12302603926802D90E090932101809320012091200130912101A5E0B0E00E943926802D0D
S123028090E0982F8827820F931F9093210180932001A6E0B0E00E943926802D90E0909361
S12302A00101809300012091000130910101A7E0B0E00E943926802D90E0982F8827820F73
S12302C0931F9093010180930001A1E0B0E00E943926802D80931E05A8E0B0E00E94392621
S12302E0802D80931301A9E5B1E00E943926802D80932A01A2E0B4E00E943926902D892F8F
S12303008150843078F080912A01843039F481E08093180183E68093D00506C082E08093B6
S1230320180102C090931801A9E0B0E00E943926802D80931201AEE0B0E00E943926802DE9
S123034080932301ABE0B0E00E943926802D80931901ACE0B0E00E943926802D80931A0174
S1230360AFE6B1E00E943926802D80931B01A2EFB1E00E943926802D80938C0580918C0560
S1230380882319F081E080938C05ADE0B0E00E943926802D26E0829FC0011124909315017F
S12303A080931401A1E7B1E00E943926802D8093F405A0E7B1E00E943926802D8093F2056E
S12303C08AE08093250681E080932306AFE8B1E00E943926802D80932B0180912B0181FF02
S12303E005C080912B01827F80932B0180912B0185FF05C080912B018F7280932B01A4EF21
S1230400B1E00E943926802D24E1829FC00111249093C9058093C805A5EFB1E00E94392686
S1230420802D8093C505A6EFB1E00E943926802D8093C305A7EFB1E00E943926802D809397
S1230440C205A8EFB1E00E943926802D90E09093C1058093C0052091C0053091C105A9EF35
S1230460B1E00E943926802D90E0982F8827820F931F9093C1058093C005ABEFB1E00E9482
S12304803926802D90E090932F0180932E0120912E0130912F01ACEFB1E00E943926802D9C
S12304A090E0982F8827820F931F90932F0180932E01ADEFB1E00E943926802D90E090930C
S12304C03101809330012091300130913101AEEFB1E00E943926802D90E0982F8827820F7A
S12304E0931F9093310180933001AFEFB1E00E943926802D90E09093330180933201209112
S1230500320130913301A0E0B2E00E943926802D90E0982F8827820F931F9093330180935C
S1230520320120E030E0D901A25ABE4F0E943926802DF901EE5DFC4F8083D901AE58BE4F63
S12305400E943926802DF901EF52FA4F8083D901A458BE4F0E943926802D808B2F5F3F4FAA
S12305602A30310501F7A7E0B2E00E943926802D80933601A3E0B2E00E943926802D809308
S1230580370120E030E0F901EE5FF94F84E6808BD901A45EBD4F0E943926802D80832F5FE4
S12305A03F4F2031310579F720E030E0D901A759BE4F0E943926802DF901EB5DFE4F80837B
S12305C02F5F3F4F2430310589F720E030E0D901A25DBD4F0E943926802DF901EE50FB4FCC
S12305E080832F5F3F4F2031310589F7ADE6B1E00E943926802D80932201A1EFB1E00E9406
S12306003926802D80938B05A0EFB1E00E943926802D80932901A6E0B2E00E943926802D56
S12306208093240120E030E0D901AA54BC4F0E943926802DF901E45DFC4F80832F5F3F4F38
S12306402031310589F7A7ECB3E00E943926802D80933901A8ECB3E00E943926802D809386
S12306603A01A4EDB3E00E943926802D80939205A5EDB3E00E943926802D80939305A6EDAE
S1230680B3E00E943926802D80939405A7EDB3E00E943926802D80939505A8EEB3E00E941C
S12306A03926802D90E090932D0180932C0120912C0130912D01A9EEB3E00E943926802D84
S12306C090E0982F8827820F931F90932D0180932C01AAEEB3E00E943926802D80938E05DD
S12306E012BC11BC089580911E0190911F01A2E0B0E0082E0E94462680911E0190911F0186
S1230700892F9927A3E0B0E0082E0E9446268091200190912101A4E0B0E0082E0E94462639
S12307208091200190912101892F9927A5E0B0E0082E0E9446268091000190910101A6E0B4
S1230740B0E0082E0E9446268091000190910101892F9927A7E0B0E0082E0E9446268091A8
S12307601301A8E0B0E0082E0E94462680911201A9E0B0E0082E0E94462612BC11BC08954C
S123078080E0A1EFB1E0082E0E9446268AE0A0EFB1E0082E0E94462680918C05A2EFB1E0FE
S12307A0082E0E94462684E0A9E5B1E0082E0E94462685E0ACE0B0E0082E0E94462682E300
S12307C0AFE6B1E0082E0E94462624E1A1E7B1E0022E0E94462691E0A0E7B1E0092E0E94ED
S12307E0462688ECA4EFB1E0082E0E944626A5EFB1E0092E0E944626A6EFB1E0022E0E944B
S123080046268AE5A7EFB1E0082E0E94462688EEA8EFB1E0082E0E94462683E0A9EFB1E020
S1230820082E0E94462680912E0190912F01ABEFB1E0082E0E94462680912E0190912F01DF
S1230840892F9927ACEFB1E0082E0E9446268091300190913101ADEFB1E0082E0E944626A6
S12308608091300190913101892F9927AEEFB1E0082E0E9446268091320190913301AFEFBE
S1230880B1E0082E0E9446268091320190913301892F9927A0E0B2E0082E0E9446268CED9F
S12308A0A7E0B2E0082E0E94462686EEA3E0B2E0082E0E9446262CE132E088ECD901082E67
S12308C00E9446262F5F3F4F82E02C323807A9F782E2AFE8B1E0082E0E94462681E0A6E094
S12308E0B2E0082E0E94462612BC11BC0895CF92DF92EF92FF920F931F93CF93DF93C0E03A
S1230900D0E0A5E0B2E00E943926202D30E040E050E0A3EDB3E00E943926602D6E01CC0C66
S1230920DD1C8CE393E0C80ED91EF601E080F18070E080E090E00E94AA2500E010E0A80139
S123094097010E94AA2524E630E040E050E00E94FC2579018A01CA01B90124EF31E040E08F
S123096050E00E94AA2528EC30E040E050E0E20EF31E041F151FA80197010E94FC25CA0137
S1230980B9012FEF30E040E050E00E94AA2525E030E040E050E00E94FC2582E0220F331F9D
S12309A0441F551F8A95D1F7CA01B90124E630E040E050E00E94FC25F601318320832196BE
S12309C0C732D10509F09DCFC0E0D0E0A9ECB3E00E943926202D30E040E050E0A3EDB3E096
S12309E00E943926602D6E01CC0CDD1C8AE893E0C80ED91EF601E080F18070E080E090E08B
S1230A000E94AA2500E010E0A80197010E94AA2524E630E040E050E00E94FC2579018A01AD
S1230A20CA01B90124EF31E040E050E00E94AA2528EC30E040E050E0E20EF31E041F151F7C
S1230A40A80197010E94FC25CA01B9012FEF30E040E050E00E94AA2525E030E040E050E0B5
S1230A600E94FC2512E0220F331F441F551F1A95D1F7CA01B90124E630E040E050E00E945B
S1230A80FC25F601318320832196C732D10509F09DCFC0E0D0E0AAECB3E00E943926202D31
S1230AA030E040E050E0A3EDB3E00E943926602D6E01CC0CDD1C88ED93E0C80ED91EF60135
S1230AC0E080F18070E080E090E00E94AA2500E010E0A80197010E94AA2524E630E040E0F4
S1230AE050E00E94FC2579018A01CA01B90124EF31E040E050E00E94AA2528EC30E040E04C
S1230B0050E0E20EF31E041F151FA80197010E94FC25CA01B9012FEF30E040E050E00E94A0
S1230B20AA2525E030E040E050E00E94FC25A2E0220F331F441F551FAA95D1F7CA01B90152
S1230B4024E630E040E050E00E94FC25F601318320832196C732D10509F09DCFC0E0D0E0DB
S1230B60A4E0B2E00E943926202D30E040E050E0A3EDB3E00E943926602D6E01CC0CDD1CBC
S1230B8086E294E0C80ED91EF601E080F18070E080E090E00E94AA2500E010E0A80197013E
S1230BA00E94AA2524E630E040E050E00E94FC2579018A01CA01B90124EF31E040E050E095
S1230BC00E94AA2528EC30E040E050E0E20EF31E041F151FA80197010E94FC25CA01B9014B
S1230BE02FEF30E040E050E00E94AA2525E030E040E050E00E94FC25E2E0220F331F441F32
S1230C00551FEA95D1F7CA01B90124E630E040E050E00E94FC25F601318320832196C73265
S1230C20D10509F09DCFDF91CF911F910F91FF90EF90DF90CF900895EAE7F0E01082109207
S1230C407C0080E880BF87EE808311B888E790E0909321058093200508950F931F93CF9379
S1230C60DF93282F30E0F901EE0FFF1FEE5FFE4F0081118143E0033F140718F0E2E3F0E0B8
S1230C804CC053E00F3D150718F0EAE0F0E045C0C0E0D0E087E290E0A901489F9001499FCF
S1230CA0300D589F300D1124D901AC0FBD1FAA0FBB1FA45CBC4F8D919C9111978017910759
S1230CC030F5FE013197E20FF31FEE0FFF1FE45CFC4F20813181608171814D915C91FE018B
S1230CE0EE0FFF1FEE0FFF1FEC0FFD1F3596201B310BC901880F991F880F991F641B750BFA
S1230D00820F931F0E94D525E60FF71F06C02196C732D10549F6E8ECF0E0CF01DF91CF9116
S1230D201F910F9108959C0180911E0584FF1BC022533040C901E3E0880F991FEA95E1F77B
S1230D40220F331F280F391F2455354F442737FD4095542F60E579E784E090E00E941E262A
S1230D60822F90E0089580911E0585FD03C084E690E0089522533040C90163E0880F991F80
S1230D806A95E1F7220F331F280F391F2455354F442737FD4095542F60E579E784E090E0F9
S1230DA00E941E262C592695822F90E008950F931F93CF93DF93AC01E0E0F0E0EF01CC0F1B
S1230DC0DD1FDE01AC58BB4F8D919C91119748175907C0F56D917C913197EE0FFF1FDF01F1
S1230DE0AC58BB4F8D919C911197681B790B8D919C91C457DB4F28813981E457FB4F0081EE
S1230E001181481B590B84E690E0DC014A9FC0014B9F900D5A9F900D11240E94D525201BEB
S1230E20310B0190F081E02D629FC001639F900D729F900D112464E670E00E94D5256E0F6C
S1230E407F1F09C03196EA30F10509F0B7CF6091A0047091A104CB01DF91CF911F910F91AA
S1230E6008950F931F93CF93DF93AC018091B4049091B5044817590718F4E0EFF0E057C0D8
S1230E808091D0049091D1048417950718F4E0E0F0E04DC0E1E0F0E0EF01CC0FDD1FDE015C
S1230EA0AC54BB4F8D919C91119748175907C0F56D917C913197EE0FFF1FDF01AC54BB4FE5
S1230EC08D919C911197681B790B8D919C91EE52FB4F20813181CE52DB4F08811981481B1C
S1230EE0590B84E690E0DC014A9FC0014B9F900D5A9F900D11240E94D525201B310B019033
S1230F00F081E02D629FC001639F900D729F900D112464E670E00E94D525E61BF70B07C00B
S1230F203196EE30F10509F0B7CFEEEFF0E0CF01DF91CF911F910F91089580911E019091C8
S1230F401F0190931D0180931C0180919305209130053091310590E08F5B9F4F82179307FB
S1230F605CF480919305882339F080917F059091800550E041E013C08091930520913005B2
S1230F803091310590E0C2968217930734F480919305882311F051E001C050E040E080918B
S1230FA09205209136053091370590E0C2968217930774F480919205882351F084EC99E0CD
S1230FC090931D0180931C0180917F059091800580919405209134053091350590E0C2960A
S1230FE08217930754F480919405882331F084EC99E090931D0180931C0180919505209146
S123100032053091330590E0C2968217930754F480919505882331F084EC99E090931D01B8
S123102080931C01442311F086E903C0552321F082E380937B05089510927B050895A895C8
S123104082E50E94F02483E10E94F02480917F0590918005892F99270E94F02480917F0557
S1231060909180050E94F02480913605909137050E94F02480913005909131050E94F0245E
S123108080912005909121050E94F02480912E0590912F050E94F02480912C0590912D0535
S12310A00E94F02480912805909129050E94F02480918505909186056091180170E00E94F0
S12310C0D525CB010E94F024809184050E94F024809183050E94F024209100063091010672
S12310E08091CC059091CD05E3E096958795EA95E1F78170232F3327822B0E94F0248091A5
S12311000006909101060E94F0248091F9059091FA050E94F02480919C050E94F024809189
S12311202605909127050E94F0248091CE059091CF05969587950E94F02483B1869586953D
S1231140817090E0909339058093380583B18695817090E090933B0580933A0580910205FC
S12311609091030590933D0580933C058091F5059091F60590933F0580933E0520919B0554
S123118030E0220F331FF901E05DFA4F80819181892F990F990B93E0220F331F9A95E1F724
S12311A0822B0E94F024E0919B05F0E0EE0FFF1FE05DFA4F808191810E94F0248DEA0E9464
S12311C0F02480919B058F5F80939B05883010F010929B050895CF92DF92EF92FF920F9388
S12311E01F93CF93DF93A89588E10FB6F89480936000109260000FBE0E943C25882309F481
S12312006AC50E94CD2490939A05809399058236910509F4E8C28336910508F041C08035A3
S1231220910509F45AC381359105E8F48534910509F4D1C08634910568F48932910509F4FB
S12312409DC48134910509F48DC08832910509F040C571C48634910509F446C18D34910566
S123126009F037C5BDC18535910509F4EAC38635910548F48235910509F4ABC3833591056A
S123128009F027C5CDC48835910509F422C48136910509F442C08735910509F01AC594C3D1
S12312A08936910509F4CAC28A369105C8F48536910509F408C28636910548F48336910545
S12312C009F494C28436910509F003C504C58636910509F4E7C08736910509F0FAC4D5C246
S12312E08037910509F4FEC28137910548F48D36910509F434C18F36910509F0EAC401C444
S12313008937910509F45DC48A37910509F471C28837910509F0DDC46CC281E60E94F02494
S123132080EA0E94F02410929A05109299050EC0EE5BFE4F80810E94F0248091990590911D
S12313409A05019690939A0580939905E0919905F0919A05E03AF10558F382E30E944124EA
S12313608EE9B7C410929A0510929905C0E0D0E00E943C25882341F1C0919905D0919A05D7
S1231380C03AD10589F40E94CD2490939A05809399058E3B910519F4C6E1DAEF15C0809134
S12313A099050E94F024FBCF0E94CD24CE5BDE4F88838091990590919A05019690939A054F
S12313C080939905C0E0D0E021964AEFC030D40708F081C4CDCFC0E0D0E00E943C25882376
S12313E009F459C00E94CD248A3B910509F073C488E10FB6F89480936000109260000FBEB9
S123140010929A05109299053EC0885B0E94F0248DEF0E94F0242091990530919A058AEF56
S123142090E0289FE001299FD00D389FD00D112407C0DE010E943926802D0E94F024219641
S12314402091990530919A052F5F3F4F8AEF90E0AC01249FC001259F900D349F900D11249D
S123146021503040C817D90720F3822F885B80950E94F0248091990590919A05019690932D
S12314809A05809399058091990590919A058430910508F4BACF21965AEFC030D50708F0F6
S12314A01AC49BCF86E60E94F02480EA0E94F02410929A05109299050EC0EE51FE4F8081C2
S12314C00E94F0248091990590919A05019690939A0580939905E0919905F0919A05E03A90
S12314E0F10558F389E9F5C310929A051092990500E010E00E943C25882349F1C091990555
S1231500D0919A05C03AD10591F40E94CD2490939A0580939905893B910519F406E11AEF15
S123152016C0E0919705F0919805099510C00E94CD24CE51DE4F88838091990590919A05DF
S1231540019690939A058093990500E010E00F5F1F4F8AEF0030180708F0BDC3CBCF8DE684
S12315600E94F02489E00E94F02480911E0190911F010E94F02480911E0190911F01892F42
S123158099270E94F02480912001909121010E94F0248091200190912101892F99270E9417
S12315A0F02480910001909101010E94F0248091000190910101892F99270E94F0248091B4
S12315C013010E94F024809112010E94F024AAE0B0E00E943926802D0E94F02482E979C33E
S12315E010929A0510929905C0E0D0E00E943C258A3008F461C00E94CD2490931F01809353
S12316001E0100911E0110911F010E94CD24982F8827800F911F90931F0180931E010E94D7
S1231620CD24909321018093200100912001109121010E94CD24982F8827800F911F90935C
S12316402101809320010E94CD24909301018093000100910001109101010E94CD24982FD5
S12316608827800F911F90930101809300010E94CD24809313010E94CD24809312010E942A
S1231680CD24AAE0B0E0082E0E9446260E94A71E0E94CD24823B910551F40E947303E091DC
S12316A09705F09198050995CFE6DAEF05C0E0919705F0919805099521964AEFC030D40707
S12316C008F009C393CF85E60E94F02483E10E94F02410929A05109299050EC0EE5DFC4FC0
S12316E080810E94F0248091990590919A05019690939A0580939905E0919905F0919A0587
S1231700EA30F10558F3809119010E94F02480911A010E94F02483E00E9442248091250105
S12317200E94F024809126010E94F024809127010E94F024809128010E94F02480911401FC
S12317409091150166E070E00E94D525CB010E94F024809122010E94F024AEE6B1E00E94E9
S12317603926802D0E94F0248AE90E94F0248CE60E94F02484E10E94F02410929A05109254
S123178099050EC0EF52FA4F80810E94F0248091990590919A05019690939A05809399051F
S12317A0E0919905F0919A05EA30F10558F310929A05109299050EC0EF52FA4F80890E9417
S12317C0F0248091990590919A05019690939A0580939905E0919905F0919A05EA30F10539
S12317E058F383E976C20E94860075C20E94C10072C20E941F086FC20E94CD24C82FD0E0CC
S12318000E94CD24C817D90709F065C20E94CD248C0190939A05809399050E94CD2408170D
S1231820190709F058C20E94CD248639910509F052C280919905CE5BDE4F4DC00E943C2567
S12318408530D0F6FBCF0E94CD24C82FD0E00E94CD24C817D90709F03EC20E94CD248C019A
S123186090939A05809399050E94CD240817190709F031C20E94CD248839910509F02BC263
S123188080919905CE51DE4F26C00E943C258530D0F6FBCF0E94CD24C82FD0E00E94CD244E
S12318A0C817D90709F017C20E94CD248C0190939A05809399050E94CD240817190709F035
S12318C00AC20E94CD248F3A910509F004C280919905CE57DD4F8883FEC10E943C25853005
S12318E0C8F6FBCFC0E0D0E00E943C25823080F10E94CD240E94CD248F38910509F0EBC1BE
S123190010929A05109299051CC0EE57FD4F108180E70E94F02482E00E94F0248091990560
S12319200E94F024812F0E94F0248FE80E94F0248091990590919A05019690939A0580937F
S12319409905E0919905F0919A05E03AF105E8F221965AEFC030D50709F4BDC1C5CF0E944F
S1231960CD248C010E94CD24F82EEE24E00EF11E0E94CD248C0190939A05809399050E94E8
S1231980CD240817190709F0A6C10E94CD24883A9105A9F4D7010E944126E070809199054B
S12319A090919A05E82BF92BF0939A05E0939905D7010F010E94522612BC11BC8CC1E0919E
S12319C09705F091980509950E943C25853038F6FBCFCC24DD240E943C25833040F10E9481
S12319E0CD24EC010E94CD248C010E94CD248D3A910509F070C1102F00270C0F1D1FD80135
S1231A000E943926F02C84E50E94F02483E00E94F0248F2D0E94F024802F0E94F024012F66
S1231A201127802F0E94F0248BEA0E94F0240894C11CD11C80E0C8168AEFD80609F44BC1D6
S1231A40CACFCC24DD240E943C258330C0F10E94CD24EC010E94CD247C010E94CD248A3AAA
S1231A60910509F038C1FE2CEE24EC0EFD1ED7010E943926802D90E0D70111960E94392613
S1231A80002D10E0102F0027080F191F85E50E94F02484E00E94F024802F0E94F024012FA1
S1231AA01127802F0E94F0248E2D0E94F024EF2CFF248E2D0E94F0248AEA0E94F02408949F
S1231AC0C11CD11C40E0C4164AEFD40609F403C1BACFC0E0D0E00E943C25882359F00E94F8
S1231AE0CD24873A910509F0F6C0E0919705F0919805099521965AEFC030D50709F4EBC0AE
S1231B00EACFC0E0D0E00E943C25882369F00E94CD248039910509F0DEC00E94FD00E09128
S1231B209705F0919805099521968AEFC030D80709F4D1C0E8CFC0E0D0E00E943C25882307
S1231B40B1F00E94CD24873D910509F0C4C080912C0590912D05ADE6B1E0082E0E94462679
S1231B6012BC11BCE0919705F0919805099521964AEFC030D40709F4AEC0DFCFC0E0D0E0D9
S1231B800E943C258823B1F00E94CD24863D910509F0A1C080912C0590912D05AEE6B1E0F2
S1231BA0082E0E94462612BC11BCE0919705F0919805099521965AEFC030D50709F48BC065
S1231BC0DFCFC0E0D0E00E943C25823010F10E94CD24892B09F07FC00E94CD2486389105E7
S1231BE0C1F489E70E94F02485E00E94F0248FEC0E94F0248FE30E94F0248EE00E94F0246E
S1231C0085E60E94F0248BE00E94F02486E80E94F02421968AEFC030D80709F45CC0D3CFA0
S1231C20C0E0D0E00E943C25823008F44CC00E94CD24892B09F047C00E94CD248C3A91055D
S1231C4009F049C083E50E94F02488E00E94F02480913C0690913D060E94F02480913C0682
S1231C6090913D06892F99270E94F0248091FC059091FD050E94F0248091FC059091FD05AE
S1231C80892F99270E94F02480912C0690912D060E94F02480912C0690912D06892F9927B6
S1231CA00E94F02480912F06909130060E94F02480912F0690913006892F99270E94F0244C
S1231CC08CEA0E94F02421964AEFC030D40719F0A9CF0E94F024A895DF91CF911F910F9185
S1231CE0FF90EF90DF90CF9008950F931F93CF93DF9310920106109200060E9439243C9A19
S1231D003D9A3F9A3E9A449A459A479A469A38984098399841983A9842983B98439838983D
S1231D2039983A983B9854985C9855985D9854985598239A269A279A2B9A2E982F98259A3F
S1231D40249A5398529822985698219820980E944424AAE5B1E00E943926802D80938D0556
S1231D600E94551E0E94A71E0E9427240E941C060E9477042B9A2E98A7E0B0E00E94392672
S1231D80802D12BC11BC85FF9BC080910001909101019F7D90930101809300010E94730376
S1231DA00E94C0030E94C1000E9486000E94FD0086E0AAE0B0E0082E0E94462689E1ABE0D7
S1231DC0B0E0082E0E9446268EE1ACE0B0E0082E0E944626AEE0B0E0082E0E94462620E0FA
S1231DE030E0F901EE5DFC4F8081D901A25ABE4F082E0E9446262F5F3F4F2A30310589F7EB
S1231E0080912501A9E6B1E0082E0E94462680912601AAE6B1E0082E0E944626809127014D
S1231E20ABE6B1E0082E0E94462680912801ACE6B1E0082E0E94462620E030E0F901EF524C
S1231E40FA4F8081D901AE58BE4F082E0E9446262F5F3F4F2A30310589F720E030E0F901CD
S1231E60EF52FA4F8089D901A458BE4F082E0E9446262F5F3F4F2A30310589F78091F4056E
S1231E80A1E7B1E0082E0E944626809114019091150166E070E00E94D525ADE0B0E0062E01
S1231EA00E94462684E1ADE6B1E0082E0E94462681EEAEE6B1E0082E0E94462612BC11BCD0
S1231EC00E94E8000E9411010E949A000E946100809100019091010185FD07C080916F0083
S1231EE08B7F80936F00449A459A80912401882311F480EC01C080E48093380110921F050C
S1231F0080911401909115018D5D954030F08CED95E0909315018093140110927C0586B3D6
S1231F20866086BB78948AEA0E94F02480E00E94F02485E50E94F02489B182958695869583
S1231F40817080938F0580916E00836080936E002B9A2E9AA89580917F05909180058E3738
S1231F60910570F180917C05882351F580910006909101069F7E9093010680930006809133
S1231F806F00856080936F0080916E00836080936E002B9A81E080937C0580910006909192
S1231FA001068062909301068093000680910006909101069062909301068093000647C076
S1231FC080917C05813009F042C080917F05909180058E379105D8F580916F008D7F8093BD
S1231FE06F00809170008C7F8093700080916F008B7F80936F0080916E00836080936E0070
S123200080910006909101068F7D90930106809300068091000690910106877F90930106BF
S123202080930006389839983A983B9854985598449A459A10927C05809100069091010645
S12320409F7D909301068093000610927A0580917C058130F9F480917A058823C1F08091CF
S12320606F00826080936F008091700083608093700080916E00836080936E0080910006A8
S123208090910106886090930106809300062B9A2E9A13C010927A05449A459A10927A058A
S12320A01092B30010928605109285058091400190914101892B09F42B9840917F0550910F
S12320C080052091200130912101809100019091010180709074822B932B4817590788F4F3
S12320E0809100069091010697FD0BC080910006909101069F7B9093010680930006469AC2
S12321000AC08091000690910106906490930106809300064698F8948091870590918805C6
S12321208A5A9A4AC1F080918705909188058555954589F07894809100069091010680647B
S1232140909301068093000688EE93E090933501809334010AC07894809100069091010699
S12321608F7B9093010680930006F8948091890590918A058A5A9A4AC1F0809189059091FA
S12321808A058555954589F0789480910006909101068068909301068093000688EE93E020
S12321A090933501809334010AC0789480910006909101068F77909301068093000680910B
S12321C03401909135010B9758F02F9A80913401909135010197909335018093340101C025
S12321E02F9880911F05833009F4F3C0843018F4882371F08EC0853009F42AC2853008F413
S123220055C1863009F4E2C1873009F0DAC268C280917D0590917E058D52914008F4D4C25F
S1232220E0911F05F0E080917800909179008C7F65E070E00E94D5256D5F7F4FEE0FFF1F21
S1232240E45AFA4F7183608380911F05C82FD0E0E0911F05F0E0EE0FFF1FE05EFA4F808138
S12322609181E0911F05F0E0EE0FFF1FE45AFA4F20813181880F991F880F991F820F931F0D
S1232280880F991F6AE070E00E94D525CC0FDD1FC05EDA4F7983688310927E0510927D0567
S12322A080911F058F5F80931F0580911F05806480937C000E94EB08809120059091210506
S12322C08035910564F42091140130911501C901880F991F820F931F9695879504C0809142
S12322E014019091150190931701809316018091400190914101892B09F461C2809140014E
S123230090914101019790934101809340012B9A56C280917D0590917E058D52914008F445
S123232053C290911F0540919605842F83708450990F990F980FE92FF0E0EE0FFF1FEE5F12
S1232340FE4F808191812091780030917900820F931F969587959183808310927E0510924E
S12323607D05A89580911F05C42FD0E08130D1F48E01085F1F4F842F0E942D06000F111F21
S1232380005E1A4FF80191838083809196058823A9F480913005909131050E949306809383
S12323A026060CC08081918162E070E00E94E925CC0FDD1FC85CDA4F7983688380911F058C
S12323C08F5F80931F0580911F05806480937C00FBC180917D0590917E058D52914008F48D
S12323E0F3C1E0911F05F0E080917800909179009695879596958795EE0FFF1FE45AFA4F6D
S12324009183808380911F05C82FD0E0E0911F05F0E0EE0FFF1FE05EFA4F80819181E0913A
S12324201F05F0E0EE0FFF1FE45AFA4F20813181880F991F880F991F820F931F65E070E039
S12324400E94D525CC0FDD1FC05EDA4F7983688310927E0510927D0580911F058F5F809358
S12324601F0580911F05806480937C000E94EB08A895809196058F5F80939605843010F0BE
S12324801092960520919605922F91709295990F907E85B18F7D892B85B9220F220F220F49
S12324A0207185B18F7E822B85B98EC180917D0590917E058D52914008F486C180912401AA
S12324C0882329F1E0911F05F0E080917800909179009695879596958795EE0FFF1FE45AC4
S12324E0FA4F91838083A0911F05B0E0E0911F05F0E0EE0FFF1FE45AFA4F80819181AA0FC0
S1232500BB1FA05EBA4F11969C938E933EC0E0911F05F0E08091780090917900EE0FFF1F3E
S1232520E45AFA4F9183808380911F05C82FD0E0E0911F05F0E0EE0FFF1FE05EFA4F008195
S12325401181E0911F05F0E0EE0FFF1FE45AFA4F808191810E9431079C01220F331F280F9A
S1232560391FC80143E0880F991F4A95E1F7801B910B820F931F6AE070E00E94D525CC0F82
S1232580DD1FC05EDA4F7983688310927E0510927D0580911F058F5F80931F0580911F0535
S12325A0806480937C0020918F0589B1829586958695817030E090E02817390709F4FFC02C
S12325C0E0919705F09198050995F9C080917D0590917E058D52914008F4F6C0E0911F0547
S12325E0F0E080917800909179009695879596958795EE0FFF1FE45AFA4F9183808380918C
S12326001F05C82FD0E0E0911F05F0E0EE0FFF1FE05EFA4F80819181E0911F05F0E0EE0F6F
S1232620FF1FE45AFA4F20813181880F991F880F991F820F931F880F991F6AE070E00E9432
S1232640D525CC0FDD1FC05EDA4F798368833EC080917D0590917E058D52914008F4B4C022
S1232660E0911F05F0E080917800909179009695879596958795EE0FFF1FE45AFA4F91838A
S12326808083E0911F05F0E0EE0FFF1FE45AFA4F2081318184E190E0FC012E9FC0012F9FAB
S12326A0900D3E9F900D11240E94D70690932B0580932A0580912A0590912B0562E070E093
S12326C00E94E92570932B0560932A0510927E0510927D0580911F058F5F80931F0568C026
S12326E080917D0590917E058D52914008F46CC0E0911F05F0E08091780090917900969514
S123270087959695879590E0EE0FFF1FE45AFA4F9183808380916A0590916B0589379105C2
S12327200CF1A0911F05B0E0E0911F05F0E0EE0FFF1FE05EFA4F40815181E0911F05F0E0B4
S1232740EE0FFF1FE45AFA4F20813181CA01880F991F840F951F820F931F9695879596956A
S1232760879519C0A0911F05B0E0E0911F05F0E0EE0FFF1FE05EFA4F20813181E0911F058C
S1232780F0E0EE0FFF1FE45AFA4F80819181820F931F96958795AA0FBB1FA05EBA4F1196E5
S12327A09C938E9310927E0510927D0510921F0580911F05806480937C000E94EB08A8953C
S12327C003C081E080931F0580917D0590917E05019690937E0580937D050E949D0780913A
S12327E07F05909180058F55914008F457C0809124068F5F809324069091240680912506F6
S1232800981708F44EC01092240680912E0590912F05E0913506FF27E7FDF095EE5FF94FC6
S1232820208130E08217930734F48091220690912306890F17C080912E0590912F05E0918C
S12328403506FF27E7FDF095EE5FF94F208130E0821793074CF08091220682302CF08091DD
S1232860220681508093220680912206E0913506FF27E7FDF095EE5FF94F2089992787FD2A
S1232880909530E02817390764F4E0913506FF27E7FDF095EE5FF94F808901C081E080931A
S12328A0220680917F05909180058739910508F461C020912C0530912D058091220190E0C5
S12328C04996281739070CF055C08091C6059091C70501969093C7058093C6052091C605DC
S12328E03091C7058091C8059091C9052817390708F442C01092C7051092C60520917F05ED
S1232900309180058091C0059091C1052817390730F49091C4058091C505890F15C020912A
S12329207F05309180058091C0059091C10549968217930758F49091C4058091C30589174B
S123294028F48091C40581508093C4059091C4058091C205891718F48091C20508C09091A1
S1232960C4058091C305981738F48091C3058093C40502C01092C40580911E0582FF1BC064
S123298080917F0590918005805D9740A0F420912C0530912D058091220190E0059628175D
S12329A039074CF481E0809391058091000690910106916007C01092910580910006909122
S12329C001069E7F9093010680930006809100019091010192FF27C020917F053091800564
S12329E080912E0190912F0182179307E0F420917F053091800580913001909131012817EC
S1232A00390788F420912C0530912D058091220190E005962817390734F480910006909103
S1232A200106946005C080910006909101069B7F9093010680930006809100019091010101
S1232A4093FF37C01A9B35C020917F053091800580913201909133018217930730F48091C3
S1232A60000690910106986005C08091000690910106977F909301068093000680911E059B
S1232A8083FF0DC080917F0590918005875D964030F08091CC059091CD05886005C080913B
S1232AA0CC059091CD05877F9093CD058093CC053DC08091CC059091CD05877F9093CD05A2
S1232AC08093CC058091370120912E0530912F0590E08217930724F4809137018823B9F490
S1232AE040917F055091800520911C0130911D01809100019091010180709078822B932BD2
S1232B008417950750F480911E0580FF06C08091000690910106986005C080910006909189
S1232B200106977F9093010680930006809100019091010180FF67C080912B0180FF11C0C9
S1232B408091B905883C28F08091C4058823B9F418C09091C4058091B9058695891790F0C8
S1232B6010C080912B0182FF0DC08091B905883C48F0809100069091010696FF02C0549AA7
S1232B8001C0549880912B0184FF16C08091B905883C28F08091220618165CF12CC02091F2
S1232BA022068091B905332727FD3095869590E0821793070CF11FC080912B0186FF1CC09F
S1232BC08091B905883CC0F020917F053091800580912C0190912D018217930760F420916E
S1232BE02E0530912F0580918E0590E08217930714F4559A01C055988091B905883C28F012
S1232C001092B90502C0549855988091B9058F5F8093B9059EC91F920F920FB60F921124D3
S1232C208F939F93809136068F5F8093360680913606882309F446C0809100069091010678
S1232C409061909301068093000610927C0580910006909101069F7D90930106809300067B
S1232C6080916F008B7F80936F0080916F008D7F80936F00809170008C7F80937000809116
S1232C806E00836080936E00449A459A80910006909101068F7D9093010680930006809102
S1232CA0000690910106877F9093010680930006389839983A983B98549855981092800553
S1232CC010927F0578949F918F910F900FBE0F901F901895282F809100069091010693FDE1
S1232CE008C0223019F0203221F402C044980895459808951F920F920FB60F9211248F9382
S1232D0080912A01813019F482E08093D0058F910F900FBE0F901F9018951F938091B2056A
S1232D20882309F466C02091B2058091B205823089F4449A8091890590918A05880F991FE6
S1232D4090938A05809389058091890590918A0581600BC08091B205803269F4459A80915A
S1232D60890590918A05880F991F90938A05809389051092B20580918400909185009093B8
S1232D80BD058093BC05479A8091F7059091F805892B61F080913106882341F08091F70557
S1232DA09091F80590938B0080938A0080917F05909180058C5D954008F055C080911E056C
S1232DC081FF51C080918A0090918B0088539F4F90938B0080938A002093310680918A007E
S1232DE090918B008C509E4F9093300680932F063AC0809131068823B1F110913106123010
S1232E00A1F4809131060E946A168091870590918805880F991F90938805809387058091B5
S1232E2087059091880581600EC010913106103281F4809131060E946A16809187059091EE
S1232E408805880F991F90938805809387051093B20580912F069091300690938B0080938B
S1232E608A00109231061F9108951F920F920FB60F9211242F933F934F935F936F937F9335
S1232E808F939F93AF93BF93EF93FF930E948D162B9A7894FF91EF91BF91AF919F918F912C
S1232EA07F916F915F914F913F912F910F900FBE0F901F9018951F920F920FB60F9211244A
S1232EC02F938F939F93F8949091130190952091D005243009F1253040F4223021F12330DE
S1232EE0A8F4213009F06CC009C02731E1F1233609F451C02E3009F063C01BC09093B20038
S1232F0084E08093B100389A83E064C096BD83E085BD3A9A84E05EC09093B2002093B100A5
S1232F203B9A82E057C096BD83E085BD399A81E051C081E0809307059093B20084E0809336
S1232F40B1008091850590918605892B11F0389A3B9A80918400909185009093BB058093E8
S1232F60BA0587E137C081E08093080596BD83E085BD8091850590918605892B11F0399AE7
S1232F803A9A80918400909185009093BF058093BE058EE01FC081E0809307059093B200BF
S1232FA084E08093B1008091850590918605892B21F0389A3B9A3A9A399A2093D0050CC037
S1232FC09093B20084E08093B100389A3B9A3A9A399A83E68093D00578949F918F912F9135
S1232FE00F900FBE0F901F901895CF93DF93EC0180918C05E7E0F0E0E81BF109EE0FFF1F54
S1233000E05EFA4F8081918120918B05821B282F30E08091290190E0880F991F880F991F84
S1233020AC01429FC001439F900D529F900D112464E670E00E94D5256436710520F083E63C
S12330408093320602C060933206809132066AE00E94C92580932906809129068A301CF0C9
S123306089E08093290680917F0590918005885E934008F0B3C0109227068FEF80933506A7
S123308080912906992787FD909564E0880F991F6A95E1F78093830580917F059091800543
S12330A064E670E00E94D525655060932E0680917F0590918005845F914060F410922E06E1
S12330C0E0912E06FF27E7FDF095E55CFE4F808190E0A3C080912E068430D9F5E091830596
S12330E0F0E0EE5BFE4F2081E0912E06FF27E7FDF095E55CFE4F6081E0912E06FF27E7FD73
S1233100F095E55CFE4F808190E09093CF058093CE05E091CE05F091CF0580917F059091FB
S1233120800540912E0630E0220F331F261B3109845F91406CE94602A0011124840F951F85
S1233140AC01249FC001259F900D349F900D11243AC0E0912E06FF27E7FDF095E45CFE4F79
S12331606081E0912E06FF27E7FDF095E55CFE4F4081E0912E06FF27E7FDF095E55CFE4F25
S1233180808190E09093CF058093CE05E091CE05F091CF0580917F059091800520912E0624
S12331A070E0641B7109845F91404CE9240290011124820F931F9C01629FC001639F900DAC
S12331C0729F900D112464E670E00E94E925E60FF71FF093CF05E093CE05C7C080917F05FA
S12331E090918005875F9242E8F086E9809327068FE0809335068091290690913506829574
S1233200807F890F80938305E0918305F0E0EE5BFE4F808190E0880F991F9093CF0580934F
S1233220CE05A3C080917F0590918005885E934062E370E00E94D5256093270680912706D1
S12332406AE00E94C9258093350680912906909135068295807F890F80938305E091830564
S1233260F0E0EE5BFE4F808190E0880F991F9093CF058093CE058091350687FD39C080916D
S123328035068F30ACF5E0918305F0E0ED5BFE4F8081E0918305F0E0EE5BFE4F6081E0917F
S12332A0CE05F091CF052091270640913506861B880F992787FD909530E06AE04602A00114
S12332C01124241B350BAC01429FC001439F900D529F900D11246AE070E00E94E9257727BD
S12332E067FD70956E0F7F1F7093CF056093CE058091290687FD39C0809129068930ACF552
S1233300E0918305F0E0EE5AFE4F8081E0918305F0E0EE5BFE4F6081E091CE05F091CF0571
S12333202091320640912906861B880F992787FD909530E06AE04602A0011124241B350B08
S1233340AC01429FC001439F900D529F900D11246AE070E00E94E925772767FD70956E0F0A
S12333607F1F7093CF056093CE0580917F0590918005855F914010F46AEB66C080917F050A
S1233380909180058952934210F06DE05DC080917F059091800585569941B0F080917F0544
S12333A090918005845699416AE070E00E94D525CB01880F991F880F991F860F971F64E67A
S12333C070E00E94D52540C080917F0590918005815A9F40B0F080917F0590918005805A53
S12333E09F406AE070E00E94D525CB01E3E0880F991FEA95E1F764E670E00E94D525645194
S123340023C080917F0590918005855F914010F460E01AC080917F0590918005845F9140C8
S12334206AE070E00E94D525CB019B0173E0220F331F7A95E1F7880F991F820F931F64E651
S123344070E00E94D52567532091CE053091CF05862F992787FD9095820F931F97FF06C0EC
S12334608091CE059091CF0561E0681B20919C05245625310CF024E14091CE055091CF052F
S12334808091120190917B0540585040480F511D491B5109822F2C3E0CF48CEE282F332772
S12334A027FD3095240F351F862F992787FD9095280F391F2A3031052CF46EE472E080E037
S12334C090E013C081E0253F38072CF064E670E080E090E00AC088E592E0821B930B9C019A
S12334E0B901882777FD8095982F20918105309182052C0F3D1F40E050E00E94AA2528E030
S123350037E040E050E00E94FC25DA01C901DF91CF910895AF92BF92CF92DF92EF92FF92F5
S12335200F931F93CF93DF93EC01E0913506FF27E7FDF095EE50FB4F808190E09093F60520
S12335408093F5056091B6057091B7052091130126952695620F711D7695679580E090E0E0
S12335602AE530E040E050E00E94AA2520918105309182052C0F3D1F13E0369527951A9528
S1233580E1F740E050E00E94FC2559016A01E0913506FF27E7FDF095EE50FB4F808190E043
S12335A0B4EBEB2EF12CCC9664EB70E00E94E925E81AF90A0027F7FC0095102FEA0CFB1C81
S12335C00C1D1D1D9E0140E050E0C801B7010E94AA2522E130E040E050E00E94FC25CA01B2
S12335E0B9012AE030E040E050E00E94FC252A97CE01A0E0B0E02A9682179307A407B507E6
S123360018F48AE090E003C0CE01821B930BDF91CF911F910F91FF90EF90DF90CF90BF90A8
S1233620AF9008950F931F93CF93DF93809184009091850090933B0680933A0680918400FB
S123364090918500C29708F404C380913606882349F088EE9DEF9093060580930505109284
S1233660360666C0E0918400F0918500C0910505D09106059E0136952795CE016AE070E093
S12336800E94D525261B370BE217F307A8F481E080933906809184009091850090933D0624
S12336A080933C0680912A01823009F0D2C28091F1048093D005CDC280918400909185007E
S12336C090932D0680932C06E0918105F091820520918400309185008091F00490E02C1B15
S12336E03D0BAC01429FC001439F900D529F900D11246EE170E00E94E925CB018E0F9F1F77
S123370062E070E00E94E925709382056093810510928205109281058091840090918500D4
S12337209093060580930505109285001092840080917A05893628F480917A058F5F8093F1
S12337407A05479880917F0590918005C0910505D0910605D093FD05C093FC052091FC059A
S12337603091FD05009102051091030540E050E060E070E489E191E00E941E26CA01B90117
S12337802EE130E040E050E00E94AA2520EC30E0A901049F9001059F300D149F300D112445
S12337A02050324040E050E00E94FC253093800520937F052091A9053091AA054091A70545
S12337C05091A805C901880F991F820F931F840F951F96958795969587959093AA05809341
S12337E0A9058091A5059091A6059093A8058093A7058091A3059091A4059093A60580939D
S1233800A5058091A1059091A2059093A4058093A30580919F059091A0059093A20580939C
S1233820A10580919D0590919E059093A00580939F0580917F059091800590939E058093D4
S12338409D0580917F05909180058D5D9540D8F040919C0580919D0590919E052091A905B8
S12338603091AA05821B930B23E0429FA0011124840F951F64E0969587956A95E1F78B5A51
S123388080939C050FC084E680939C05809181059091820564E070E00E94E9257093820576
S12338A0609381051092360680917F05909180058059914060F58091020590910305049797
S12338C031F180913906813011F584E090E090930305809302058091020590910305806879
S12338E0809381001092850010928400D695C795D695C795D0930605C09305058091FC0578
S12339009091FD05969587959695879532C080917F05909180058955924078F18091020594
S123392090910305039749F180913906813029F583E090E090930305809302058091020537
S1233940909103058068809381001092850010928400CC0FDD1FCC0FDD1FD0930605C09302
S123396005058091FC059091FD05880F991F880F991F9093FD058093FC058091FC059091FA
S1233980FD050E94F5179093300680932F068091CC059091CD0583FF39C0C091B305D09118
S12339A0B405CE0163E070E00E94D525892B41F18091FC059091FD0563E070E00E94D52502
S12339C07093300660932F06E0912F06F0913006209139018091FC059091FD0568E270E06B
S12339E00E94D52530E0629FC001639F900D729F900D11248E0F9F1F9093300680932F06D7
S1233A002196D093B405C093B30504C01092B4051092B30580917F05909180058A5892405C
S1233A2018F484E690E009C080912005909121058E3691053CF488EC90E090933806809374
S1233A40370604C0109238061092370680912F069091300620911601309117014091370656
S1233A6050913806821B930B841B950B90932B0680932A0680912A0690912B0697FF20C009
S1233A8080912A0690912B062091FC053091FD0540912F0650913006820F931F8417950783
S1233AA078F42091FC053091FD0580912F0690913006821B930B449690932B0680932A06D8
S1233AC0F89480917F0590918005805E9E4208F095C0809100069091010693FD8FC08091E1
S1233AE02A0690912B068739910504F11092B20580912A0690912B0690938B0080938A00BE
S1233B0080918A0090918B009093F8058093F70580913906882311F480E201C082E0809393
S1233B2031061092B20584E090E05CC080912A0690912B068B5B9F4F2CF11092B20584E6BA
S1233B4090E090938B0080938A009093F8058093F70580913906882311F480E201C082E0F2
S1233B6080933106809131060E946A161092B20588E290E09093FA058093F90584E18093AF
S1233B80040534C080912F069091300690938B0080938A002091FC053091FD0580912A0686
S1233BA090912B06820F931F9093F8058093F70580913906882341F480E20E946A1680E227
S1233BC08093B20582E007C082E00E946A1682E08093B20580E28093310684E18093040511
S1233BE084EB90E09093FA058093F9051092390680910006909101069F770FC08091FC0598
S1233C009091FD058C509E4F90938B0080938A0080910006909101069068909301068093F5
S1233C20000680917F05909180058D549D4138F080918400909185008C599F4F06C0809173
S1233C40FC059091FD050E948A1A90938900809388007894DF91CF911F910F9108951F9235
S1233C600F920FB60F9211242F933F934F935F936F937F938F939F93AF93BF93EF93FF938C
S1233C800E94121B2B9A7894FF91EF91BF91AF919F918F917F916F915F914F913F912F9120
S1233CA00F900FBE0F901F9018951092800081EF9FEF909389008093880085EF9FEF90930D
S1233CC08B0080938A00109285001092840084E090E0909303058093020580910205909119
S1233CE0030580688093810080916F00876080936F00539852983C9A3D9A449A459AA2E092
S1233D00B2E00E943926802D8093F004A1E0B2E00E943926802D8093F1048091F1048E30CB
S1233D2039F08091F104873119F087E18093F10480918D05813021F4809169008C6003C08D
S1233D4080916900886080936900E99A089521EB30E0F90110821092B6001092B20010926B
S1233D60B300A0E7B0E08C9183608C9338984098399841983A9842983B9843983898399809
S1233D803A983B98EFE6F0E080818D7F80838C918C7F8C9386E0F901808384E68093F105A8
S1233DA00895813099F438983B9880912A01843021F439983A98109208051092410610929F
S1233DC04006109207051092B1000895823049F439983A9810923F0610923E0610920805ED
S1233DE015BC08951F920F920FB60F9211242F933F934F935F936F937F938F939F93AF9352
S1233E00BF93EF93FF93F89480910705843051F48091B20090E09093FF058093FE0581E0C5
S1233E200E94D11E7894FF91EF91BF91AF919F918F917F916F915F914F913F912F910F90E2
S1233E400FBE0F901F9018950F931F9380912005909121050A9714F487E003C0809191054B
S1233E6086E08093B1001092B20080917F0590918005845F914018F410922E0616C0809108
S1233E807F05909180058D56974020F08EE080932E060BC080917F059091800564E670E0D5
S1233EA00E94D525655060932E06E0912E06F0E0E45DFC4F8081809313018091910588230B
S1233EC029F02091F2018091180108C0E0918305F0E0EE51FE4F808120911801829FC0012D
S1233EE011249093B7058093B60580917F05909180058059914048F5809100019091010185
S1233F0082FF19C08091B6059091B70520911901820F911D9093B7058093B60580910006CC
S1233F2090910106846090930106809300068EE18093B5053FC080910006909101068B7FAA
S1233F40909301068093000635C080910006909101068B7F90930106809300068091B505CE
S1233F60823028F08091B50581508093B505E091B605F091B70580911901209119014091DA
S1233F80B505E80FF11D8EE190E0841B910930E0AC01429FC001439F900D529F900D1124A5
S1233FA06EE170E00E94D525E61BF70BF093B705E093B60580919105882309F0ABC1E0912A
S1233FC08305F0E0EE51FE4F808120911801829FC00111249093B7058093B605809135061E
S1233FE087FD3EC0809135068F30D4F5E0918305F0E0ED51FE4F6081E0918305F0E0EE512A
S1234000FE4F40810091B6051091B7058091270620913506E091180170E0641B710990E078
S12340204AE0240290011124821B930B9C01629FC001639F900D729F900D11246AE070E0B0
S12340400E94E925F0E06E9FC0016F9F900D7E9F900D1124800F911F9093B7058093B60588
S12340608091290687FD3EC0809129068930D4F5E0918305F0E0EE50FE4F6081E09183058A
S1234080F0E0EE51FE4F40810091B6051091B7058091320620912906E091180170E0641BD4
S12340A0710990E04AE0240290011124821B930BAC01649FC001659F900D749F900D1124CA
S12340C06AE070E00E94E925F0E06E9FC0016F9F900D7E9F900D1124800F911F9093B7053C
S12340E08093B605809100019091010184FF55C020914A0530914B0580912C0590912D057B
S123410028173907C4F480912C0590912D0520914A0530914B05821B930B64E070E00E944D
S1234120E92580918405861710F460938405809123018093B8053091B8053430C8F0809106
S1234140B6059091B705E0918405F0E0EE5DFC4F2081820F911D9093B7058093B605315055
S12341603093B8058091000690910106806109C0109284051092B805809100069091010609
S12341808F7E909301068093000680912C0590912D0590934B0580934A058091000190912E
S12341A0010191FFB4C080918F05882309F0AFC08091F3058F5F8093F3059091F305809111
S12341C0F405981708F4A6C01092F3058091280590912905E0912906FF27E7FDF095EF523A
S12341E0FA4F208130E028173907B4F48091280590912905E0912906FF27E7FDF095EF529D
S1234200FA4F2081821B910962E070E00E94E9256C596093F1052BC0809128059091290511
S1234220E0912906FF27E7FDF095EF52FA4F208130E082179307DCF48091F1051816BCF428
S1234240E0912906FF27E7FDF095EF52FA4F8081209128053091290590E0821B930B62E0E6
S123426070E00E94E92584E6861B8093F10580910006909101069D7F909301068093000688
S12342802091F105E0912906FF27E7FDF095EF52FA4F8089332727FD309590E08C599F4F2B
S12342A08217930754F4E0912906FF27E7FDF095EF52FA4F80898C591EC02091F105E091E2
S12342C02906FF27E7FDF095EF52FA4F4089332727FD309584E690E0841B910928173907F4
S12342E0CCF4E0912906FF27E7FDF095EF52FA4F908984E6891B8093F105809100069091D9
S123430001069260909301068093000603C084E68093F1058091B6059091B70520912606A1
S123432030E062E070E00E94E925269FC001279F900D369F900D112464E670E00E94D52561
S1234340660F771F7093B7056093B605209136053091370580911B0190E0C2962817390784
S1234360D4F5809100019091010181FF34C08091360590913705C397D4F040911A01809103
S12343801A01209136053091370560911B0190E070E06E5C7F4FFC01E29FC001E39F900D52
S12343A0F29F900D11240E94D525461B03C080911A01482F50E08091B6059091B705480F03
S12343C0591F5093B7054093B6058091000690910106826005C080910006909101068D7F03
S12343E0909301068093000680912401882371F02091B6053091B7058091F105245630405A
S1234400992787FD9095280F391F0DC02091B6053091B7058091F1052C593F4F992787FD8C
S12344209095281B390B3093B7052093B6058091CC059091CD0583FF1CC0E091B605F091FF
S1234440B70520913A018091B6059091B70564E170E00E94E92530E0629FC001639F900D51
S1234460729F900D11248E0F9F1F9093B7058093B605809100019091010190FF4CC080916C
S1234480200590912105823891050CF044C08091B6059091B70520912501820F911D90937A
S12344A0B7058093B605E0912005F0912105609118012091250182E890E08E1B9F0B70E0D3
S12344C0AB01849FB001859F700D949F700D11248FEF90E0FB01E89FB001E99F700DF89F14
S12344E0700D1124882777FD8095982F30E040E050E00E94AA2520E43FE140E050E00E9420
S1234500FC258091B6059091B705820F931F9093B7058093B6052091B6053091B7058091E3
S1234520180145EF849FC00111248217930754F480911801849FC00111249093B705809361
S1234540B6050BC08091B6059091B7051816190624F01092B7051092B605809100069091D4
S1234560010692FF05C0109286051092850510C020918505309186058091B6059091B70581
S1234580820F931F96958795909386058093850540917F055091800520911C0130911D01DA
S12345A0809100019091010180709078822B932B4817590730F480910006909101069F7727
S12345C00DC080911E0580FD04C010928605109285058091000690910106906890930106DB
S12345E08093000678941F910F9108951F920F920FB60F9211242F933F934F935F936F934E
S12346007F938F939F93AF93BF93EF93FF93F89420910705223039F0243009F44FC0213013
S123462009F051C01CC080914006909141068F3F9105D1F1C8F180914006909141068F5F45
S12346408093B30080914006909141068F5F904090934106809340062093070534C00E94FB
S1234660241F8091850590918605909341068093400680914006909141068F3F9105A1F035
S123468098F080914006909141068F5F8093B30080914006909141068F5F90409093410634
S12346A08093400682E007C080914006909141068093B30084E08093070505C081E00E94A4
S12346C0D11E109207057894FF91EF91BF91AF919F918F917F916F915F914F913F912F91CD
S12346E00F900FBE0F901F9018951F920F920FB60F9211242F933F934F935F936F937F93E6
S12347008F939F93AF93BF93EF93FF93F89420910805223039F0243009F453C0213009F026
S123472053C020C080913E0690913F068F3F910591F088F080913E0690913F068F5F87BD7D
S123474080913E0690913F068F5F904090933F0680933E0633C080913E0690913F0687BD2B
S123476084E024C0809185059091860590933F0680933E0624E025BD16BC80913E069091B9
S12347803F068F3F9105A9F0A0F080913E0690913F068F5F87BD80913E0690913F068F5FAD
S12347A0904090933F0680933E0682E0809308050BC080913E0690913F0687BD209308055A
S12347C003C082E00E94D11E7894FF91EF91BF91AF919F918F917F916F915F914F913F9173
S12347E02F910F900FBE0F901F9018951F920F920FB60F9211242F933F934F935F936F9337
S12348007F938F939F93AF93BF93EF93FF93F89480910805843049F486B590E09093CB054D
S12348208093CA0582E00E94D11E7894FF91EF91BF91AF919F918F917F916F915F914F91C3
S12348403F912F910F900FBE0F901F90189554985C9855985D985498559815BCEEE6F0E04D
S123486080818360808384E085BD16BC82E187BD089511B88FEF84B915B887B98AB9089520
S1234880089508950895089588E98093C10083E18093C40089E896E090934706809346066A
S12348A0909343068093420689E496E090934506809344069093CA068093C90610924806BA
S12348C01092FB0508951F920F920FB60F9211248F939F93EF93FF9380914806882311F134
S12348E0E0914606F091470681918093C600F0934706E0934606E95CF64030F089E896E02D
S123490090934706809346068091480681508093480680914806882329F48091C1008F7D2E
S12349208093C100FF91EF919F918F910F900FBE0F901F9018951F920F920FB60F921124EB
S12349402F938F939F93EF93FF938091C600E091C906F091CA0680838091FB058F5F8093AC
S1234960FB058091C9069091CA0601969093CA068093C9068958964030F089E496E0909319
S1234980CA068093C906FF91EF919F918F912F910F900FBE0F901F9018958091FB0588231E
S12349A019F48FEF9FEF0895F8948091FB0581508093FB05E0914406F09145062191F09300
S12349C04506E0934406E958F64030F089E496E090934506809344067894822F90E00895BC
S12349E0982F809148068F33E0F780914806803418F080E090E00895F894809148068F5F93
S1234A0080934806E0914206F091430690838091420690914306019690934306809342067A
S1234A20895C964030F089E896E090934306809342068091C10080628093C100789481E0F4
S1234A4090E00895CF93DF93EC0104C00E94F0248111219688818823C9F781E090E0DF910C
S1234A60CF91089589E095E00E942225089581E195E00E94222508958091FB0590E0089556
S1234A80CF92DF92EF92FF920F931F93CF93DF93CDB7DEB729970FB6F894DEBF0FBECDBFE6
S1234AA08C01F62EE42EDE011196E4E1F5E089E001900D928150E1F749E06E010894C11CBC
S1234AC0D11CFF2081F089E090E0841B91092F2D30E08217930738F04150F601E40FF11DF3
S1234AE08CE28083FF244150F601E40FF11DC8016AE070E00E94D525805D8083C8016AE0A3
S1234B0070E00E94D5258B01672B11F4FF2019F085E08F15B0F619E01E197E010894E11C63
S1234B20F11C07C0F701E10FF11D80810E94F0241F5F1930B8F329960FB6F894DEBF0FBE04
S1234B40CDBFDF91CF911F910F91FF90EF90DF90CF900895629FD001739FF001829FE00D49
S1234B60F11D649FE00DF11D929FF00D839FF00D749FF00D659FF00D9927729FB00DE11D3B
S1234B80F91F639FB00DE11DF91FBD01CF0111240895991B79E004C0991F961708F0961BE5
S1234BA0881F7A95C9F780950895AA1BBB1B51E107C0AA1FBB1FA617B70710F0A61BB70B94
S1234BC0881F991F5A95A9F780959095BC01CD01089597FB092E07260AD077FD04D0E5DFA5
S1234BE006D000201AF4709561957F4F0895F6F7909581959F4F0895A1E21A2EAA1BBB1B2E
S1234C00FD010DC0AA1FBB1FEE1FFF1FA217B307E407F50720F0A21BB30BE40BF50B661F9E
S1234C20771F881F991F1A9469F760957095809590959B01AC01BD01CF01089597FB092EFC
S1234C4005260ED057FD04D0D7DF0AD0001C38F450954095309521953F4F4F4F5F4F08959B
S1234C60F6F790958095709561957F4F8F4F9F4F0895F999FECFB2BDA1BDF89A119600B4BE
S1234C800895F7DFE02DF5DFF02D0895F999FECFB2BDA1BD00BC11960FB6F894FA9AF99AFB
S1234CA00FBE0895F3DF012CF1DF11240895FFCF2F000100020003000400050006000700CC
S1234CC008003228E803900106141E3C401F401F6419121E01010203040A0411C409C4094F
S1234CE08813AC0D6400DCE64003020A14324696500054819596B7AFC3C8BEBEB9B0AFAF41
S1234D00ADAC4984C0CBD2D6D7D0C7C2BBB8B3AEAAA9458AA2A9AAB7C0BABEBBB6B8B2B39E
S1234D20B4B93281868DA4A58B8C8F9EA6A2A6A5A6C034525D5B596F788285858281FF8525
S1234D409FB034444E4B4A54615769727272737D9095272C1B252B334B5155616A6D6C7DC2
S1234D60828B1D211A242A32454C4F5E6169717E818634323232323232323232327F323241
S1234D80323232323232323232323232323232323232131718191B1C1D1F21232527282CD9
S1234DA02E311418191A1C2124272B3035393C3E414316191D232A31353B3F42484E565AE1
S1234DC05E651B1D363E525863666C6E777D84898D932226434B6172818A9097A8ACAFB163
S1234DE0B6B9292E484E6B7C939BA2AFB9BFCBD2D2D229344B536E7F9CA8B1BCC5D0D2D262
S1234E00D2D2283F4E587187A4B2BAC2D2D2D2D2D2D23746545E7691B1BEC4D2D2D2D2D2A4
S1234E20D2D239485660869FBAD2D2D2D2D2D2D2D2D2000000000000000000000000000052
S1234E4000000000000000000000000000000000000000000000000000000000000000004E
S1234E600000000000000000000000000000000000000102030405060708090A0B0C0D0EC5
S1234E800F100102030405060708090A0B0C0D0E0F100102030405060708090A0B0C0D0EFE
S1234EA00F1014161718191A1B1C1D1E1F2021222324191A1B1C1D1E1F202122232425264F
S1234EC027271E1F2022232425262728292A2B2C2D2E000204060708090A0C0E282624223F
S1234EE0201E1E1E1E1E1E1E1E1E1E1EF0FF80BBE0880465484BA438022BF0207019CC1335
S1234F00860F440CC209D0074C061B052A046A03D1025602F201A1015F012801FB00D600DF
S1234F20B7009D0087007500660059004D0044003C0034002E0029002500F0FF80BBE0884F
S1234F400465484BA438022BF0207019CC13860F440CC209D0074C061B052A046A03D10269
S1234F605602F201A1015F012801FB00D600B7009D0087007500660059004D0044003C000A
S1234F8034002E0029002500F0FF80BBE0880465484BA438022BF0207019CC13860F440C69
S1234FA0C209D0074C061B052A046A03D1025602F201A1015F012801FB00D600B7009D00D0
S1234FC087007500660059004D0044003C0034002E0029002500F0FF80BBE0880465484B07
S1234FE0A438022BF0207019CC13860F440CC209D0074C061B052A046A03D1025602F2017A
S1235000A1015F012801FB00D600B7009D0087007500660059004D0044003C0034002E0052
S1235020290025000000F5047E05AE066C08C00AB30D630F8B10D7118813000000000A0056
S12350400F001E003C007800FA007201E00180028002000008000A000C000E00C80A4A06CB
S12350607E0484031A002000270032003E0066008E00B202EB02240337034B035603610351
S12350807003E800D600C200B0009D008A00780078006500520040002D001900070000000E
S12350A001175A5A5A5050505050505050505050505003003200FA04041B5B481B5B324ACF
S11150C0000D0A0020202020202020202000A7
S503028773
